:100D0D007580F875E18F75E9C875908075E27F750E
:100D1D00EA8075A0E075E33F75EBC075B01975E419
:0B0D2D00E675EC194380C043E980220A
:080DB500E4F5A8F5A9F5AA2256
:100D5E0075C432E4F587759850759D7F759C6475E2
:0C0D6E009E04439D80759A0A759BFF222D
:090DAC00120DB5120D0DC200225A
:100C370053B1F8120DACE4F51B7FFF7E0FFDFC12DC
:100C47000D94EF645A7026C201751D55120D385068
:100C5700028005120D385005E4F51D8024E4F51DCA
:100C6700758E55438702000000000080F0E4F51BF5
:100C77007FFF7E0FFDFC120D94BFA505D201020078
:050C8700A6121000227E
:100A1B00E4F508F509900202F0900205740BF090D2
:100A2B000203E0FFA3E0900203F0A3EFF07F02903C
:100A3B000202E0FE2407FDE433FCEFC39DEC64806F
:100A4B00F8748098501774002FF582E43402F58304
:100A5B00E02509F509E43508F5080F80D274072E57
:100A6B00F582E43402F583E509F0E508FF90020214
:100A7B00E02408F582E43402F583EFF0C202E4F5DA
:100A8B0086C29C7400252BF582E43402F583E0F5D5
:010A9B0099C1
:010A9C002237
:100CD500E4900206F0A3E0FFB4490FA3E0B4410A93
:100CE500A3E0B45005C201D20022EFB4491190022D
:100CF50008E0B4530AA3E0B45005D201D200229013
:080D05000206740AF0C200228C
:10045000E4F526F525F524F523F530F52FF52EF5F1
:100460002DF52AF529F528F527900209E0FFE4FC8F
:10047000FDFE781012073CC004C005C006C007A3EB
:10048000E0FFE4FCFDFE781812073CD003D002D058
:1004900001D000EF4BFFEE4AFEED49FDEC48FCC0F9
:1004A00004C005C006C007900208E0FFE4FCFDFEA2
:1004B000780812073CD003D002D001D000EF4BFBEC
:1004C000EE4AFAED49F9EC48F8900207E0FFEB4FED
:1004D000F52AEAF529E9F528E8F527200006900233
:1004E00006740AF0E4FF7E78FDFCAB2AAA29A9284D
:1004F000A827D312071840052001028017E4FF7EC9
:10050000ECFDFCAB2AAA29A928A827D3120718407A
:100510000A3001079002067401F022E4900206F00E
:10052000F521751D55F515FF7E0EFDFC120B7EE4C1
:10053000F515FF7E0EFDFC120C8C502B30012E7534
:100540001BA5E4F51C7FFF7E0FFDFC120B15E4F5E7
:100550001B7FFF7E0FFDFC120D94EF64A5600E90D3
:1005600002067403F080069002067402F0E4F51DA2
:10057000900206E06003020631FB7A02F9F8AF2A26
:10058000AE29AD28AC271206868F09E4F508E508E8
:10059000C395094003020637E4F50A300107F50E5A
:1005A000750D108006E4F50E750D84F50CF50BE560
:1005B0000825E0FEE4FCFD250EF50EE50D3EF50DEB
:1005C000ED350CF50CEC350BF50B300135E5092458
:1005D000FEFBE434FFFAED34FFF9EC34FFF8AF082A
:1005E000E4FED3120718501A750A01E5082402FF29
:1005F000C3EF9509FFEF25E0FEE4F50E8E0DF50C37
:10060000F50B751D55AF0EAE0DAD0CAC0B850A1577
:10061000120B7EAF0EAE0DAD0CAC0B850A15120C95
:100620008C40069002067402F0E4F51D05080205F0
:070630008E9002067405F034
:0106370022A0
:10089500D203E4F510F511AE10AF11E4FCFDFB7ABF
:1008A50002F9F8D3120718500302098CE4F5163043
:1008B500015E2526F515E5253410F514E43524F5F6
:1008C50013E43523F512E4252AFFE529340CFEE46B
:1008D5003528FDE43527FCAB15AA14A913A812C3C6
:1008E5001207184040E4252AFBE529340CFAE435C3
:1008F50028F9E43527F8C3E5159BF515E5149AF5B0
:1009050014E51399F513E51298F51275160180157E
:10091500E42526F515E5253484F514E43524F51389
:10092500E43523F512AF15AE14AD13AC12740025E2
:1009350011F58274003510F583E0F51B85161C1240
:100945000B15AF15AE14AD13AC1285161B120D9415
:1009550074002511F58274003510F583E06F60048D
:10096500C2038023E5262401F526E43525F525E493
:100975003524F524E43523F5230511E5116003023B
:09098500089C051002089CA20365
:01098E002246
:1001F100C200900206E0FFC395214014E5212404CA
:10020100FDE433FCD3EF9DEC6480F8748098400AE0
:10021100900206E060047405F022900206E0F521E8
:10022100E4F0900202E070152526F526E52534025A
:10023100F525E43524F524E43523F52322E521547D
:1002410003F50AE4F508F509900202E0FD7C00C31C
:10025100E5099DE5089C503274072509F582E434CF
:1002610002F583E0FBAF0A7E00120638E5092FFF95
:10027100E5083EFE74002FF58274003EF583EBF035
:100281000509E50970C2050880BEE50A640360033B
:1002910002044F751D551208955003020386E4FFB1
:1002A1007E02FDFCAB26AA25A924A823120718402B
:1002B1001AE5269400F526E5259402F525E5249412
:1002C10000F524E5239400F5238009E4F526F525BE
:1002D100F524F523E4F50F30015E2526F50EE5251D
:1002E1003410F50DE43524F50CE43523F50BE42544
:1002F1002AFFE529340CFEE43528FDE43527FCAB63
:100301000EAA0DA90CA80BC31207184040E4252A18
:10031100FBE529340CFAE43528F9E43527F8C3E57F
:100321000E9BF50EE50D9AF50DE50C99F50CE50B17
:1003310098F50B750F018015E42526F50EE525349A
:1003410084F50DE43524F50CE43523F50B751D55C5
:10035100AF0EAE0DAD0CAC0B850F15120B7EAF0EB3
:10036100AE0DAD0CAC0B850F15120C8C500E120896
:100371009540129002067403F002044C9002067438
:1003810002F002044CE4F50A75F004E50AA4240223
:10039100F582E5F03400F583E0FFE4FCFDFE781022
:1003A10012073CC004C005C006C00775F004E50A89
:1003B100A42403F582E5F03400F583E0FFE4FCFDBD
:1003C100FE781812073CD003D002D001D000EF4BC9
:1003D100FFEE4AFEED49FDEC48FCC004C005C00635
:1003E100C00775F004E50AA42401F582E5F03400A4
:1003F100F583E0FFE4FCFDFE780812073CD003D052
:1004010002D001D000EF4BFBEE4AFAED49F9EC487E
:10041100F875F004E50AA42400F582E5F03400F54E
:1004210083E0FFEB4FFFEAFEE9FDE8FCE5302FF545
:1004310030E52F3EF52FE52E3DF52EE52D3CF52D32
:0E044100050AE50A64806003020389E4F51DE4
:01044F00228A
:10098F007E007D007C00900209E0FFE478101207E2
:10099F003CC004C005C006C007A3E0FFE4FCFDFE99
:1009AF00781812073CD003D002D001D000EF4BFFD4
:1009BF00EE4AFEED49FDEC48FCC004C005C006C080
:1009CF0007900208E0FFE4FCFDFE780812073CD018
:1009DF0003D002D001D000EF4BFBEE4AFAED49F9FC
:1009EF00EC48F8900207E0FFEB4FFFEAFEE9FDE865
:1009FF00FCAB30AA2FA92EA82DC3120718600790A1
:0B0A0F0002067408F022E4900206F0DA
:010A1A0022B9
:100BDE00E4900206F0752C0A751D55F515FF7E0E74
:100BEE00FDFC120B7EE4F515FF7E0EFDFC120C8C47
:100BFE00502A200130751B5AE4F51C7FFF7E0FFD35
:100C0E00FC120B15E4F51B7FFF7E0FFDFC120D94FD
:100C1E00EF645A6010900206740380059002067409
:090C2E0002F0E4F52CE4F51D22AE
:100A9D00E4F52B900202E0FD2408F582E43402F522
:100AAD0083E0FE74072DF582E43402F583E07C00CB
:100ABD002400FFEC3EFEEF65327003EE65316003FE
:100ACD00432280E5226006900206F08038900205F0
:100ADD00E0FEB40605120CD5802BEEB4070512040A
:100AED00508022900205E0B408051201F1801690A5
:100AFD000205E0B4090512098F800A900205E0B4E1
:080B0D000A03120BDE020A1BB1
:1000A600E4F526F525F524F523F530F52FF52EF59F
:1000B6002DF52C120D5E20980302018E7400252B5F
:1000C600F582E43402F583E599F0052BE52BC3941C
:1000D6008C4003E4F52BE52BB4010D900200E0649F
:1000E6005A700302018C806BE52BB4021490020156
:1000F600E064A56002805CE4F531F532F522020188
:100106008C900202E0FF7E002409FDEE33FCAB2B4F
:100116007A00C3EB9DEC6480F87480985062EF24FB
:1001260007FFEE33FED3EB9FEE6480F874809850A1
:100136001574FF252BF582E43401F583E02532F5AD
:1001460032E43531F531E52BB4050D900204E06457
:10015600076033E4F52B802EE52B640670289002A9
:1001660005E0FF6406601FEF6407601AEF6408602D
:1001760015EF64096010EF640A600B4322308006B5
:1001860053B1F8120A9DC29830994453B1F89002BF
:1001960002E02408FFE433FEC3E52B9FEE6480F8FB
:1001A6007480984013E4F586D29CF52B900200F0FB
:1001B600A3F0A3F0D2028015052BE4F586C29C7449
:1001C60000252BF582E43402F583E0F599C299E522
:1001D6002C640A60030200BC53B1F820020302003B
:0B01E600BCC202F52C1200000200BC9D
:100B7E008F148E138D128C118515A7AF14AE13AD75
:100B8E0012AC1178081207298FF775F2E620AF3CE8
:100B9E0075F305E5A76515703375F40AE51DB455B3
:100BAE002B75F509AF14AE13AD12AC117808120700
:100BBE0029A804A905AA06AB07AFF7E4FCFDFEC3FE
:100BCE00120718700775F60600000000E4F5A7225C
:080C8C008F148E138D128C11E0
:100C9400D2048515A7E4F516F517AE16AF17E4FCD4
:100CA400FDFB7A02F9F8D3120718401FE517251443
:100CB400FFE51635138F82F583E4936004C2048044
:100CC4000A0517E51770D3051680CFE4F5A7A2042B
:010CD40022FD
:100B15008F1A8E198D188C17851CA7AF1AAE19ADB3
:100B250018AC1778081207298FF7E51AFF8FFB8590
:100B35001BFC75F26E20AF3D75F305E5A7651C70CE
:100B45003475F40AE51DB4552C75F509AF1AAE19BF
:100B5500AD18AC177808120729A804A905AA06AB91
:100B650007AFF7E4FCFDFEC3120718700875F6061B
:090B75000000000000E4F5A722D5
:080D94008F1A8E198D188C17BF
:0F0D9C00E4851BA7851A8285198393FFE4F5A7C9
:010DAB002225
:10077C00E4F50853B1F8E508C3943A501FE4F50AC0
:10078C00AF08FE7C02FD12074FE42FF510EE34107B
:10079C00F50FE43DF50EE43CF50D8021750A01AF33
:1007AC00087E007C027D0012074FE42FF510EE341A
:1007BC008CF50FED34FFF50EEC34FFF50D751D5572
:1007CC00AF10AE0FAD0EAC0D850A15120B7EAF102F
:1007DC00AE0FAD0EAC0D850A15120C8C4003020841
:1007EC0083E4F50BF50CAE0BAF0CE4FCFDFB7A02CD
:1007FC00F9F8D31207185003020886AF087E007C64
:10080C00027D0012074FA804A905AA06AB07E42530
:10081C000CFFE50B3484FEE433FDE433FCEB2FFFDB
:10082C00EA3EFEE93DFDE83CFCE4F51B120D948F1D
:10083C0009E50C2510FFE50B350FFEE4350EFDE444
:10084C00350DFC85091B850A1C120B15E50C2510B2
:10085C00FFE50B350FFEE4350EFDE4350DFC850A86
:10086C001B120D94EF650960037F0222050CE50C49
:10087C007002050B0207F27F01220508E508C394FC
:08088C003C500302077F7F00CE
:010894002241
:100D3800D20312077CEF7019F515FF7E0EFDFC1229
:100D48000B7EE4F515FF7E0EFDFC120C8C920380E1
:050D580002C203A2032A
:010D5D002273
:03000000020D7A74
:100D7A0075817F75B208000000000000000043B2D0
:0A0D8A000478FFE4F6D8FD020C37F0
:03000300021003E5
:03000B0002100BD5
:03001300021013C5
:03001B0002101BB5
:03002300021023A5
:03002B0002102B95
:0300330002103385
:03003B0002103B75
:0300430002104365
:03004B0002104B55
:0300530002105345
:03005B0002105B35
:0300630002106325
:03006B0002106B15
:0300730002107305
:03007B0002107BF5
:03008300021083E5
:03008B0002108BD5
:03009300021093C5
:03009B0002109BB5
:0300A3000210A3A5
:10063800EF8DF0A4A8F0CF8CF0A428CE8DF0A42ED6
:02064800FE2290
:10064A0075F008758200EF2FFFEE33FECD33CDCC67
:10065A0033CCC58233C5829BED9AEC99E5829840EA
:10066A000CF582EE9BFEED9AFDEC99FC0FD5F0D6C7
:10067A00E4CEFBE4CDFAE4CCF9A88222B800C1B9F1
:10068A000059BA002DEC8BF084CFCECDFCE5F0CB2F
:10069A00F97818EF2FFFEE33FEED33FDEC33FCEB68
:1006AA0033FB10D703994004EB99FB0FD8E5E4F923
:1006BA00FA227818EF2FFFEE33FEED33FDEC33FC10
:1006CA00C933C910D7059BE99A4007EC9BFCE99A04
:1006DA00F90FD8E0E4C9FAE4CCFB2275F010EF2F49
:1006EA00FFEE33FEED33FDCC33CCC833C810D70749
:1006FA009BEC9AE899400AED9BFDEC9AFCE899F884
:0E070A000FD5F0DAE4CDFBE4CCFAE4C8F92216
:10071800EB9FF5F0EA9E42F0E99D42F0E89C45F037
:0107280022AE
:10072900E8600FECC313FCED13FDEE13FEEF13FFAE
:03073900D8F122D2
:10073C00E8600FEFC333FFEE33FEED33FDEC33FC1B
:03074C00D8F122BF
:10074F00EC8EF0A4CCC5F0CCCDF8EFA4CEC5F02D37
:10075F00FDE43CFCE8A42EC8C5F03DFDE43CFCEFF5
:0D076F00A4FFE5F028FEE43DFDE43CFC2283
:00000001FF
